:100000000C9472060C94B6060C94B6060C94B606C4
:100010000C94B6060C94B6060C94B6060C94B60670
:100020000C94B6060C94B6060C94B5110C94871279
:100030000C9468200C94B6060C94B6060C94B60684
:100040000C94B6060C94B6060C94B6060C94B60640
:100050000C94B6060C94D0200C94B6060C94B606FC
:100060000C94B6060C94B6060C94B6060C94B60620
:100070000C94B6060C94B6060C94B6060C94B60610
:100080000C94B6060C94B6060C94B6060C94B60600
:100090000C94B6060C94B6060C94B6060C94B606F0
:1000A0000C94B6060C94B6060C94B606F41216130D
:1000B0000414161304145B137E130414D313E613F1
:1000C00029172917581758179717B717E718E71858
:1000D000C217E71872187218D818E718E718E1184D
:1000E0007F187F187F187F187F187F187F187F1858
:1000F0007F187F187F187F187F187F187F187F1848
:100100008F189D18A418AB18B51814001A00080011
:100110001500170000001C0018000C00120013004E
:1001200004001600070009000A0000000B000D0083
:100130000E000F0033001D001B0006001900050013
:10014000E2001100100036003700380029002B00B3
:10015000E300E1002A00E4002C0003522D003400EB
:10016000280014001A00090013000A0000000D0006
:100170000F0018001C0033000400150016001700C3
:10018000070000000B00110008000C0012001D0009
:100190001B00060019000500E2000E0010003600EA
:1001A0003700380029002B00E300E1002A00E400BA
:1001B0002C0003522D003400280034003600370094
:1001C00013001C00000009000A00060015000F00C3
:1001D00004001200080018000C00000007000B00CB
:1001E000170011001600330014000D000E001B0054
:1001F000E200050010001A0019001D0029002B0064
:10020000E300E1002A00E4002C0003522D00380036
:10021000280049004A0052004D004B000000A90090
:100220002400250026002F004C00500051004F00F4
:100230004E000000AA0021002200230030003500FB
:10024000AC00AE00AB002D00E200A8001E001F00B5
:100250002000310004546500E300E1002A00E400BE
:100260002C000100370027002E000100FB00F000E9
:10027000FC00F90000000053400041004200430030
:100280000100F200F100F300FA00000001533F000A
:100290003E003F004400F700F400F500F600F700D0
:1002A000E20002533A003B003C004500010001001F
:1002B000E300E1002A00E4002C000100010001003D
:1002C00000500A44454255473A20656E61626C65AC
:1002D000642E0A005374617465206F6620726F7714
:1002E0002025583A2025303136620A0048756D6164
:1002F0006E2D7265616461626C65206D61747269F6
:10030000782073746174653A0D0A004465626F75F4
:100310006E63696E672064656C61792072656D61DA
:10032000696E696E673A2025580A005B735D004B61
:100330006579626F6172642073746172742E0A0051
:100340005B575D005B535D005B525D005B445D008D
:100350005B435D000E034100740072006500750090
:1003600073000000180354006500630068006E000D
:100370006F006D0061006E006300790000000403EF
:10038000090409028D00050100A0FA09040000011A
:1003900003010100092111010001223F000705812D
:1003A0000308000A090401000103010200092111E8
:1003B000010001224D000705820308000A0904021A
:1003C000000103000000092111010001223600078D
:1003D00005830308000A0904030002030000000962
:1003E00021110100012220000705840320000107DC
:1003F00005040320000109040400010300000009B2
:1004000021110100012239000705850310000112A6
:1004100001100100000008EDFE6060010001020013
:100420000105010906A101050719E029E7150025C5
:1004300001950875018102050819012905950575C1
:10044000019102950175039101050719002977159E
:10045000002501957875018102C00631FF0974A15C
:10046000010975150025FF9520750881020976158B
:100470000025FF952075089102C005010980A101A2
:10048000850216010026B7001A01002AB700751070
:1004900095018100C0050C0901A101850316010029
:1004A000269C021A01002A9C02751095018100C049
:1004B00005010902A1010901A10005091901290588
:1004C00015002501950575018102950175038101CE
:1004D0000501093009311581257F950275088106CE
:1004E00009381581257F950175088106050C0A38A4
:1004F000021581257F950175088106C0C005010997
:1005000006A101050719E029E715002501950875E1
:1005100001810295017508810105081901290595D8
:1005200005750191029501750391010507190029CF
:10053000FF150025FF950675088100C00A002530CB
:10054000325820006B6579626F6172645F7265700A
:100550006F72743A20004B6579626F617264204C4F
:100560004544732073746174653A2025780A0064E9
:10057000656C5F6B65795F6269743A2063616E27B1
:10058000742064656C3A20253032580A0061646436
:100590005F6B65795F6269743A2063616E277420CE
:1005A0006164643A20253032580A00290A00257512
:1005B000002F002575005D280025640020002564BB
:1005C00000200025640020002564007C00253032D6
:1005D00058006D6F7573656B6579205B62746E7C16
:1005E000782079207620685D287265702F61636CB1
:1005F000293A205B006D6B5F776865656C5F746995
:100600006D655F746F5F6D6178203D2025640A0021
:100610006D6B5F776865656C5F6D61785F73706542
:100620006564203D2025640A006D6B5F74696D650B
:100630005F746F5F6D6178203D2025640A006D6BEB
:100640005F6D61785F7370656564203D2025640A85
:10065000006D6B5F696E74657276616C203D20255C
:10066000640A006D6B5F64656C6179203D202564D0
:100670000A006D6B5F776865656C5F74696D655FB7
:10068000746F5F6D6178203D2025640A006D6B5F9B
:10069000776865656C5F6D61785F73706565642010
:1006A0003D2025640A006D6B5F74696D655F746F32
:1006B0005F6D6178203D2025640A006D6B5F6D6180
:1006C000785F7370656564203D2025640A006D6B5A
:1006D0005F696E74657276616C203D2025640A0046
:1006E0006D6B5F64656C6179203D2025640A000AAA
:1006F00000257500363A20776865656C5F74696D12
:10070000655F746F5F6D61783A20000A002575009F
:10071000353A20776865656C5F6D61785F737065E9
:1007200065643A20000A00257500343A2074696D2A
:10073000655F746F5F6D61783A20000A002575006F
:10074000333A206D61785F73706565643A20000A02
:1007500000257500323A20696E74657276616C28E6
:100760006D73293A20000A00257500313A2064652E
:100770006C6179282A31306D73293A20000A092DDD
:100780002056616C756573202D0A004D3E004D2585
:10079000643E20003F007365742064656661756C7B
:1007A000740A00433E200077686572652064656CBA
:1007B00074613A20637572736F723D25642C2077E3
:1007C0006865656C3D25640A5365652068747470BE
:1007D0003A2F2F656E2E77696B6970656469612E9B
:1007E0006F72672F77696B692F4D6F7573655F6BDC
:1007F0006579730A000A092D204D6F7573656B6565
:1008000079202D0A4553432F713A09717569740A8D
:10081000313A0964656C6179282A31306D73290A8F
:10082000323A09696E74657276616C286D73290AB3
:10083000333A096D61785F73706565640A343A090B
:1008400074696D655F746F5F6D61780A353A097719
:100850006865656C5F6D61785F73706565640A36A5
:100860003A09776865656C5F74696D655F746F5F81
:100870006D61780A0A703A097072696E7420766147
:100880006C7565730A643A09736574206465666102
:10089000756C74730A75703A092B310A646F776E40
:1008A0003A092D310A706775703A092B31300A7098
:1008B00067646F776E3A092D31300A0A7370656587
:1008C00064203D2064656C7461202A206D61785F2E
:1008D0007370656564202A202872657065617420D4
:1008E0002F2074696D655F746F5F6D6178290A00F0
:1008F0003F004D3E2000433E20004C25640A00741A
:10090000696D65725F636F756E743A202530346C63
:10091000580A006B6579626F6172645F6E6B726F0B
:100920003A2025580A006B6579626F6172645F69CD
:10093000646C653A2025580A006B6579626F6172B4
:10094000645F70726F746F636F6C3A2025580A0091
:10095000686F73745F6B6579626F6172645F6C65F9
:10096000647328293A2025580A000A092D20537457
:1009700061747573202D0A004743433A20342E39A1
:100980002E32204156522D4C4942433A20312E38C6
:100990002E31204156525F415243483A20617672CF
:1009A000350A004F5054494F4E533A204C5546415A
:1009B000204D4F5553454B45592045585452414BB6
:1009C000455920434F4E534F4C4520434F4D4D41C9
:1009D0004E44204E4B524F20343039360A00425597
:1009E000494C443A20313637313865662D64697296
:1009F0007479202832333A30393A3131204A756ED1
:100A00002020392032303136290A005649443A2014
:100A100030784645454428546563686E6F6D616E55
:100A2000637929205049443A2030783630363028CE
:100A300041747265757329205645523A20307830DA
:100A40003030310A00444553433A20712E6D2E6BED
:100A50002E206B6579626F617264206669726D77B2
:100A600061726520666F72204174726575730A0049
:100A70000A092D2056657273696F6E202D0A000ACF
:100A8000092D20436F6E736F6C65202D0A4553430B
:100A90002F713A09717569740A6D3A096D6F757332
:100AA000656B65790A000A092D204D61676963202D
:100AB0002D0A443A094465627567204D6573736178
:100AC000676520546F67676C650A583A094D617411
:100AD000726978204465627567204D6F64652054A3
:100AE0006F67676C65202D2053686F77206B657981
:100AF0007072657373657320696E206D61747269BD
:100B00007820677269640A4B3A094B6579626F61B4
:100B1000726420446562756720546F67676C652056
:100B20002D2053686F77206B657970726573732021
:100B30007265706F72740A4D3A0944656275672078
:100B40004D6F75736520546F67676C650A563A0977
:100B500056657273696F6E0A533A095374617475FE
:100B6000730A433A09416374697661746520436F7F
:100B70006E736F6C65204D6F64650A46312D46318A
:100B8000303A0953776974636820746F204C617937
:100B9000657220302D392028463130203D204C30E0
:100BA000290A302D393A0953776974636820746FC4
:100BB000204C6179657220302D390A4553433A093A
:100BC00053776974636820746F204C617965722073
:100BD000302028616C7465726E617465206B657974
:100BE0002031290A47524156453A095377697463BF
:100BF0006820746F204C6179657220302028616C08
:100C00007465726E617465206B65792032290A50B3
:100C1000415553453A094A756D7020746F20426FF3
:100C20006F746C6F616465722028526573657429F6
:100C30000A4E3A094E4B524F20546F67676C650A53
:100C4000003F004E4B524F3A206F66660A004E4BF3
:100C5000524F3A206F6E0A000A6D6F7573653A2025
:100C60006F66660A000A6D6F7573653A206F6E0ACB
:100C7000000A6B6579626F6172643A206F66660A7A
:100C8000000A6B6579626F6172643A206F6E0A00C8
:100C90000A6D61747269783A206F66660A000A6D9F
:100CA00061747269783A206F6E0A000A6465627531
:100CB000673A206F66660A000A64656275673A20C3
:100CC0006F6E0A000A0A4A756D70696E6720746F4C
:100CD00020626F6F746C6F616465722E2E2E20001F
:100CE000433E200011241FBECFEFDAE0DEBFCDBFB0
:100CF00004B603FE24C08091FE019091FF01A091F3
:100D00000002B09101028730904BA740B04BB9F47C
:100D10001092FE011092FF01109200021092010247
:100D200014BE84B7877F84BF88E10FB6F8948093A0
:100D30006000109260000FBEE0E0F8E3099511E05A
:100D4000A0E0B1E0E8E4F3E502C005900D92A8341C
:100D5000B107D9F711E0A8E4B1E001C01D92AE3FA0
:100D6000B107E1F70E94EF0E0C94A2290C94000049
:100D7000FF93EF93E0914801F0914901309709F01A
:100D80000995EF91FF910895FC018591803011F054
:100D9000EFDFFBCF0895FF27E0E230E247FF0CC012
:100DA000419597FF09C0EDE260957095809590950B
:100DB000611D711D811D911D27FF02C0219530E32A
:100DC00050E2AA27660F771F881F991FAA1FA41732
:100DD00010F0A41B63955A95A9F7AA3008F0A95FF3
:100DE000A05DAF93F395611571058105910541F7FC
:100DF000ED3211F4EF93F395F21718F43F93F39556
:100E0000FBCF8F91B5DFFA95E1F70895E991F9915C
:100E10008591803021F0853219F0AADFF9CF08954D
:100E200020E0E89455915532C1F3503311F46894A1
:100E300055915A3348F4505390F3220F022E220F4B
:100E4000220F200D250FF4CF0EF421958991999151
:100E5000533619F3533729F1533559F1BC0188271B
:100E60009927E8945C3621F4899199916894559179
:100E7000543639F446EF7EF077FF0DC08FEF9FEFC9
:100E80000AC055374AE039F0583540E121F0523672
:100E900042E009F00895FF93EF937DDFEF91FF911A
:100EA000B7CFFF93EF93FC0181918030B9F360DFFE
:100EB000FBCFFF93EF9368DFF1CFDF93CF93CDB7F5
:100EC000DEB72596A3DFCF91DF91089508950895A9
:100ED00086E697E0892B11F00C946607089587E663
:100EE00097E0892B11F00C946707089561110BC0EE
:100EF000FC018281882321F085EE0E94CD1503C07C
:100F000085EE0E94951680E090E0089581E00895B6
:100F100081E008950C94880708950F931F93CF9351
:100F2000DF938C01FC01C081D181CE010E944B1E58
:100F3000BE010E943A08EC01B8010E948A0788238A
:100F400009F48DC0F8018281882309F44AC0809198
:100F5000550181111FC0C431F0E5DF0709F051C010
:100F60000E948C0781E0809355010E949A20909303
:100F700054018093530110924C0110924E01109233
:100F80004D011092500110924F0110925201109297
:100F9000510165C080915301909154010E94A62097
:100FA000883C910570F480914C01E82FF0E0EE0F41
:100FB000FF1FE35BFE4FD183C0838F5F80934C01A3
:100FC0004EC0C43880E5D80721F0C538D04501F1BE
:100FD0003AC0F8018281882341F010924A0182E0F0
:100FE0001EC0C438E0E5DE0759F580914A01811141
:100FF00006C086E20E94CD1586E20E94951682E028
:101000001CC0C438F0E5DF0741F3C538D045D9F43A
:10101000F8018281882331F010924B0180E20E9416
:10102000E4161DC080914B01811106C087E20E9429
:10103000CD1587E20E94951680E20E94EB160FC044
:10104000C538D04529F381E080934A0180934B0154
:10105000C801DF91CF911F910F910C94860780E01A
:10106000DF91CF911F910F9108950C9468070C9414
:101070006F0708959BE0799FF00111249CE2899FFE
:10108000E00DF11D1124E60FF11DEE0FFF1FE65FCD
:10109000FE4F859194910895880F991FFC01E657A2
:1010A000F040859194910895880F991FFC01E65FA7
:1010B000FE4F8591949108950F931F93CF93DF93E3
:1010C000EC01811520E3920750F5C11580E2D807A5
:1010D00008F0C9C0CB3BD10590F4C83AD10508F05F
:1010E00070C0C53AD10508F061C0C430D10508F020
:1010F000DAC1219709F0D4C101E010E014C2CF3F5A
:10110000D10511F008F0CFC1C03FD10508F0A8C04B
:10111000CE01805E9109089708F4C5C1C1C1C130F4
:1011200090E5D90709F4A8C050F5C0318FE4D8077D
:1011300070F4C11590E4D90708F09AC0C11521E3F5
:10114000D20708F0ADC1DD278E01106CECC1C115CE
:10115000D04509F0A5C10E9452198FEF94E32CE00D
:10116000815090402040E1F700C0000087E797E7FA
:1011700090930108809300080E94F520D4C1C11506
:1011800097E5D90758F4C03121E5D20708F020C10E
:10119000C43180E5D80708F479C082C1CE019057E8
:1011A0008115904108F07CC1DF7077C1C53AD10547
:1011B00009F47BC1C63AD10509F07AC102E810E40E
:1011C000B2C1C83AD10509F476C1C93AD10509F4CA
:1011D00075C1CA3AD10509F474C1CB3AD10509F4F5
:1011E00073C1CC3AD10509F472C1CD3AD10509F4E5
:1011F00071C1C03BD10509F470C1CE3AD10509F4E3
:101200006FC1CF3AD10509F46EC1C13BD10509F4D4
:101210006DC1C23BD10509F46CC1C33BD10509F4D2
:101220006BC1C43BD10509F46AC1C53BD10509F4C2
:1012300069C1C63BD10509F468C1C73BD10509F4B2
:1012400067C1C83BD10509F466C1C93BD10509F4A2
:1012500065C1CA3BD10509F464C100E014E463C16F
:101260008E01106560C1CE019F700E9454085CC160
:10127000DF708E01106A57C182EC92E00E94C406B2
:101280008091DF0181608093DF014DC10E944C217C
:10129000811102C00E9432210E945F2190E0909350
:1012A000FE018093FD01C23080E5D80721F48091D2
:1012B000FD01816086C0C43090E5D90721F480919A
:1012C000FD0182607EC0C63020E5D20721F4809106
:1012D000FD01846076C0C83080E5D80719F480919C
:1012E000FD0127C0CA3090E5D90721F48091FD01A6
:1012F000806167C0CC3020E5D20721F48091FD01E8
:1013000080625FC0CE3080E5D80721F48091FD0176
:10131000806457C0C03190E5D90721F48091FD0168
:1013200080684FC0C23120E5D20729F48091FD01C9
:101330008460886046C0C33080E5D80721F480917E
:10134000FD018E7F3EC0C53090E5D90721F4809124
:10135000FD018D7F36C0C73020E5D20721F4809192
:10136000FD018B7F2EC0C93080E5D80719F480912C
:10137000FD0126C0CB3090E5D90721F48091FD0115
:101380008F7E1FC0CD3020E5D20721F48091FD0172
:101390008F7D17C0CF3080E5D80721F48091FD0103
:1013A0008F7B0FC0C13190E5D90721F48091FD01F9
:1013B0008F7707C0C331D04531F48091FD018B7F19
:1013C000877F8093FD018091FD010E946321ABC066
:1013D0008D2F99278F70992781309105D9F49E011F
:1013E0002370332702C0880F991F2A95E2F79C6863
:1013F0008E0144E0000F111F4A95E1F7002713709A
:10140000802B912B53E0CC0FDD1F5A95E1F7C0766E
:10141000DD272FC08230910531F4DC2FCC278E01DF
:10142000016F106A80C08330910569F4CE0183702A
:10143000992701E010E002C0000F111F8A95E2F722
:10144000C8019C680FC084309105B9F4CE01837047
:10145000992701E010E002C0000F111F8A95E2F702
:10146000C8019A6823E0CC0FDD1F2A95E1F7C07E02
:10147000D7708C010C2B1D2B56C08530910531F493
:10148000DC2FCC278E01046F106A4DC0069709F03F
:101490004AC0CF71DD27DC2FCC278E01106243C0FC
:1014A00000E010E040C08E013EC001E810E43BC007
:1014B00003E810E438C002EE14E435C009EE14E489
:1014C00032C00AEE14E42FC005EB14E42CC006EB86
:1014D00014E429C007EB14E426C00CEC14E423C088
:1014E0000DEC14E420C003E815E41DC00AE815E47F
:1014F0001AC002E915E417C004E915E414C001E2BA
:1015000016E411C003E216E40EC004E216E40BC0B8
:1015100005E216E408C006E216E405C007E216E498
:1015200002C00AE216E4C801DF91CF911F910F912A
:1015300008959BE0799FF00111249CE2899FE00DC2
:10154000F11D1124E60FF11DEE0FFF1FE65FFE4FA8
:1015500085919491803E9105E0F4803C910558F589
:101560008133910509F46FC048F48932910509F47B
:1015700063C08A32910509F46DC072C08933910548
:10158000E9F082389105D1F08533910509F44DC019
:1015900067C0833E910581F138F4803E9105B9F032
:1015A000823E9105D9F05CC0863E910561F1873E8F
:1015B0009105A1F155C00E944C0808952091FD01AC
:1015C00020FD02C021FF4CC080EE90E049C0809118
:1015D000FD0180FFF9CF89E390E042C08091FD01D9
:1015E00082FF0EC08091FD0184FF03C080E090E087
:1015F00037C083EE90E034C08091FD0182FFF2CFCE
:1016000082EE90E02DC08091FD0183FF0BC08091A0
:10161000FD0184FDEBCF87EE90E022C08091FD01BB
:1016200083FFF5CF86EE90E01BC08091FD0185FF22
:1016300007C089E290E014C08091FD0185FFF9CFD9
:1016400085E390E00DC08091FD0186FF07C08AE22E
:1016500090E006C08091FD0186FFF9CF81E390E024
:101660000E945C08089508950C94330BE82FF0E075
:10167000E05EFE4F8081E82FEF70F0E082958F7082
:1016800021E030E0A90102C0440F551F8A95E2F71E
:1016900040A308950F931F93CF93DF9385B780687E
:1016A00085BF85B7806885BFC3E0D0E001E010E06A
:1016B000FE01E05EFE4F8081E82FEF70F0E021A197
:1016C00082958F70A80102C0440F551F8A95E2F7DA
:1016D000CA01822B81A38C2F0E94360B219740F7E1
:1016E0008AE090E061E070E0FC01EB5EFE4F20815B
:1016F000E22FEF70F0E042A122952F70DB0102C0D3
:10170000AA0FBB1F2A95E2F79D01242B22A3019764
:1017100058F7DF91CF911F910F910C943508EF92FC
:10172000FF920F931F93CF93DF930EE511E0C3E079
:10173000EE24E394F12CD5E08C2F0E94360B8AE046
:1017400090E040E050E0FC01EB5EFE4F6081E62F50
:10175000EF70F0E020A130E062956F7002C0359527
:1017600027956A95E2F720FD09C09701082E02C06F
:10177000220F331F0A94E2F7422B532B019718F7DD
:10178000F801929182918F018417950721F051837E
:101790004083D09300018C2F0E94360BC15060F61D
:1017A0008091000187FD42C09091DF0190FF10C041
:1017B000282F332727FD30953F938F938BE093E0BD
:1017C0009F938F930E945D070F900F900F900F9043
:1017D0008091000181508093000187FD07C08FE94F
:1017E0009FE00197F1F700C0000020C080915C01EC
:1017F00090915D01909365018093640180915A01FD
:1018000090915B01909363018093620180915801F4
:1018100090915901909361018093600180915601EC
:101820009091570190935F0180935E010E94370869
:1018300081E0DF91CF911F910F91FF90EF9008957C
:10184000E82FF0E0EE0FFF1FE25AFE4F80819181FA
:101850000895EF92FF920F931F93CF93DF938091A0
:10186000DF0180FF04C08CEE92E00E94C4060EE50A
:1018700011E0C0E0D0E084EDE82E82E0F82E809107
:10188000DF0180FF13C0F801808191810E940F2049
:101890009F938F93DF93CF93FF92EF920E945D0708
:1018A0000F900F900F900F900F900F9021960E5F5A
:1018B0001F4FC430D10519F7DF91CF911F910F91C0
:1018C000FF90EF9008950F931F93CF9306E611E0DA
:1018D000C0E0F801929182918F010E94ED1FC80F24
:1018E000F1E00E351F07A9F78C2FCF911F910F91B3
:1018F00008958091790108959FB7F8941092680136
:101900009FBF9091F401943009F057C09091E90085
:101910009F703091EC00232F217030FD20E8922B36
:1019200024E02093E9002091EB0020FF43C02091A8
:10193000EE0027FF3FC020916601222321F0209175
:10194000E80025FF37C01092660126E03091E800DC
:1019500035FD15C03091F401343061F53091EB0064
:1019600035FD28C0215021F481E08093660122C01A
:10197000EFE9FFE03197F1F700C00000E7CF809377
:10198000F1008091E80085FD0AC08091E80080FFA9
:10199000FCCF8091E8008E778093E80006C08FB777
:1019A000F89421E0209368018FBF9F709093E90025
:1019B00080E008959F709093E9008FEF0895CF9392
:1019C000DF9300D01F92CDB7DEB79C018091F40168
:1019D000843019F593E099833B832A839093E9003F
:1019E0008FEF9091E800815095FD06C095ED9A9596
:1019F000F1F700008111F5CF8091E80085FF0DC05F
:101A000040E050E063E070E0CE0101960E94A50F37
:101A10008091E8008E778093E8000F900F900F90F0
:101A2000DF91CF910895CF93DF9300D01F92CDB770
:101A3000DEB72091F401243021F522E029839B8335
:101A40008A8383E08093E9008FEF9091E8008150D2
:101A500095FD06C095ED9A95F1F700008111F5CF3F
:101A60008091E80085FF0DC040E050E063E070E049
:101A7000CE0101960E94A50F8091E8008E77809399
:101A8000E8000F900F900F90DF91CF910895209173
:101A9000F4012430F1F422E02093E9002FEF30919B
:101AA000E800215035FD06C035ED3A95F1F700000C
:101AB0002111F5CF2091E80025FF0BC040E050E058
:101AC00065E070E00E94A50F8091E8008E7780931A
:101AD000E8000895CF93DF932091F401243009F0BA
:101AE00048C0EC0180910B018823E1F080910C014A
:101AF0008823C1F085E08093E9008FEF9091E800A2
:101B0000815095FD06C095E19A95F1F7000081118D
:101B1000F5CF8091E80085FF2CC040E050E060E107
:101B200070E017C081E08093E9008FEF9091E800AA
:101B3000815095FD06C095ED9A95F1F70000811151
:101B4000F5CF8091E80085FF14C040E050E068E0E8
:101B500070E0CE010E94A50F8091E8008E778093FF
:101B6000E80080E1FE01A9E6B1E001900D928A95BE
:101B7000E1F7DF91CF91089580E593E00E94C406DC
:101B80008091F301811109C00E943A110E949711BE
:101B90008091E20084608093E20008958CE493E0F9
:101BA0000E94C4061092F301089588E493E00C9417
:101BB000C40684E493E00C94C40680E493E00E949D
:101BC000C4060C946220209167012F5F822F62E38C
:101BD0000E943229992319F02093670108951092E9
:101BE000670180916801882371F18091F40184304C
:101BF00041F58091E9008F702091EC00922F917057
:101C000020FD90E8892B94E09093E9009091EB00FF
:101C100090FF14C09091EE0097FF10C09091E800E3
:101C200095FF03C01092F100F9CF9091E80090FF6A
:101C300005C09091E8009E779093E8008F708093A4
:101C4000E90010926801089542E061EC81E00E9491
:101C5000B41042E061EC82E00E94B41042E061EC1A
:101C600083E00E94B41042E261EC84E00E94B41070
:101C700042E161EC85E00C94B4108091F601833070
:101C800009F455C030F4813071F0823009F48EC00F
:101C900008958A3009F47AC08B3009F460C0893025
:101CA00009F09CC020C08091F501813A09F096C0EE
:101CB0008091E800877F8093E8008091F9019091FE
:101CC000FA01892B21F460E189E691E003C060E02C
:101CD00080E090E070E00E94F00F8091E8008B7748
:101CE0008093E80008958091F501813209F076C073
:101CF0008091F9019091FA01009719F0049709F089
:101D00006DC08091E800877F8093E8008091E800B3
:101D100082FD05C08091F4018111F8CF5FC08091F0
:101D2000F100809379018091E8008B7753C0809116
:101D3000F501813A09F052C08091F9019091FA01C0
:101D4000892B09F04BC08091E800877F8093E800E1
:101D50008091E80080FFFCCF80910B0136C080911C
:101D6000F5018132D9F58091F9019091FA01892B21
:101D7000A9F58091E800877F8093E8000E94E91030
:101D80008091F70180930B010C9452198091F50119
:101D9000813221F58091E800877F8093E8000E94DE
:101DA000E9108091F80180937A0108958091F501FE
:101DB000813AA1F48091E800877F8093E8008091C8
:101DC000E80080FFFCCF80917A018093F100809140
:101DD000E8008E778093E8000C94E910089584B7AA
:101DE000877F84BF88E10FB6F894809360001092DB
:101DF00060000FBE90E080E80FB6F8948093610019
:101E0000909361000FBE0E94C9140E943A110E9473
:101E100097118091E20084608093E2008CE79CE05F
:101E20000E94E81F78940E941C140E94CB1481E049
:101E300091E00E9437148FE293E00E94C4068091E3
:101E4000F401853089F48BE293E00E94C4060E947D
:101E500029208091F201882391F30E945420882345
:101E600071F30E948F0FEBCF0E94EF14E8CF292F60
:101E7000332723303105C9F064F42130310581F076
:101E80002230310509F043C08DE890E022E833E0CC
:101E900042C021323105F1F02232310541F137C023
:101EA00082E190E02FE034E036C09927813091053F
:101EB00041F08230910541F0892B49F5EEE7F3E0DE
:101EC00005C0E4E6F3E002C0E4E5F3E0849190E0CD
:101ED0009F0121C06530D8F4E62FF0E0EE0FFF1F20
:101EE000ED5CFE4F2081318189E090E014C06530C7
:101EF00070F470E0FB01EE0FFF1FE75DFE4F2081E5
:101F00003181FB01EC5DFE4F808190E004C080E0F8
:101F100090E020E030E0FA0131832083089580E1F1
:101F200089BD82E189BD09B400FEFDCF8091D80052
:101F30008F7D8093D8008091E00082608093E000E4
:101F40008091E00081FDFCCF0895CF92DF92EF9267
:101F5000FF920F931F93CF93DF93EC018B016A01E4
:101F60000E940811811133C0C114D10439F0F60167
:101F700080819181081B190BC80FD91FE12CF12C0E
:101F80000115110519F18091E80085FD16C08091B9
:101F9000E8008E778093E800C114D10449F0F6017F
:101FA00080819181E80EF91EF182E08285E00FC008
:101FB0000E940811882321F30AC089918093F100BF
:101FC00001501109FFEFEF1AFF0ADACF80E0DF912D
:101FD000CF911F910F91FF90EF90DF90CF900895D8
:101FE0002091FB013091FC012617370748F061155D
:101FF000710539F42091E8002E772093E80001C0A4
:10200000B90140E061157105A9F12091F401222385
:1020100009F443C0253009F442C02091E80023FDB3
:1020200040C02091E80022FD32C02091E80020FF4E
:10203000E9CF4091F3002091F20030E0342BFC0115
:10204000CF016115710559F02830310540F48191B7
:102050008093F100615071092F5F3F4FF1CF41E054
:102060002830310509F040E02091E8002E772093D8
:10207000E800C8CF4111C9CF0AC08091F40188237C
:1020800061F0853061F08091E80083FD0AC08091A5
:10209000E80082FFF2CF80E0089582E0089583E0B7
:1020A000089581E008952091FB013091FC012617ED
:1020B000370748F06115710539F42091E8002E7753
:1020C0002093E80001C0B901FC0120E06115710511
:1020D00091F18091F401882309F440C0853009F41E
:1020E0003FC08091E80083FD3DC08091E80082FD03
:1020F0002FC08091E80080FFE9CF2091F30080910C
:10210000F20090E0922B6115710559F0883091052D
:1021100040F424912093F1003196615071090196A9
:10212000F2CF21E0089709F020E08091E8008E7757
:102130008093E800CBCF2111CCCF0AC08091F4016D
:10214000882361F0853061F08091E80083FD0AC04A
:102150008091E80082FFF2CF80E0089582E0089548
:1021600083E0089581E00895982F973058F5909373
:10217000E900981739F07091EC002091ED00509132
:10218000F00003C0242F762F50E021FF19C03091BA
:10219000EB003E7F3093EB003091ED003D7F3093BC
:1021A000ED003091EB0031603093EB007093EC0068
:1021B0002093ED005093F0002091EE0027FF07C020
:1021C0009F5FD3CF8F708093E90081E0089580E016
:1021D00008958091F50187FF11C08091E80082FD8C
:1021E00005C08091F4018111F8CF11C08091E80001
:1021F0008B770BC08091F401882349F08091E8002F
:1022000080FFF8CF8091E8008E778093E8000895F2
:102210002091E4003091E50095E64091EC00842F98
:10222000817040FF22C08091E80080FD1CC0809139
:10223000F401882391F0853091F08091EB0085FDC9
:1022400010C04091E4005091E5004217530729F374
:102250009A01915011F784E0089582E0089583E097
:10226000089581E0089580E008954091E80042FFDC
:10227000DECF08950E94A8110E94B011E0EEF0E0B8
:10228000808181608083E8EDF0E080818F778083BA
:1022900019BCA7EDB0E08C918E7F8C9380818F7EEE
:1022A00080831092F30108950F931F93CF93DF93D0
:1022B0000E94A8110E94B011C8EDD0E088818F77EC
:1022C000888388818068888388818F7D888319BC12
:1022D0001092F4011092F0011092F2011092F101AB
:1022E00000EE10E0F80180818B7F8083888181601F
:1022F000888342E060E080E00E94B410E1EEF0E00C
:1023000080818E7F8083E2EEF0E080818160808337
:10231000808188608083F80180818E7F80838881BE
:1023200080618883DF91CF911F910F910895E8ED2F
:10233000F0E080818F7E8083E7EDF0E08081816036
:10234000808384E082BF81E08093F3010C94541178
:10235000E8EDF0E080818E7F80831092E2000895A6
:102360001092DA001092E10008951F920F920FB6BA
:102370000F9211242F933F934F935F936F937F930B
:102380008F939F93AF93BF93EF93FF938091E1005F
:1023900082FF0BC08091E20082FF07C08091E100C4
:1023A0008B7F8093E1000E94E30D8091DA0080FF33
:1023B0001FC08091D80080FF1BC08091DA008E7F03
:1023C0008093DA008091D90080FF0DC080E189BD43
:1023D00082E189BD09B400FEFDCF81E08093F40164
:1023E0000E94BC0D05C019BC1092F4010E94CE0DD4
:1023F0008091E10080FF19C08091E20080FF15C04C
:102400008091E2008E7F8093E2008091E200806103
:102410008093E2008091D80080628093D80019BC3C
:1024200085E08093F4010E94D90D8091E10084FF42
:1024300030C08091E20084FF2CC080E189BD82E140
:1024400089BD09B400FEFDCF8091D8008F7D8093B7
:10245000D8008091E1008F7E8093E1008091E200BE
:102460008F7E8093E2008091E20081608093E200A1
:102470008091F001882311F084E007C08091E3008F
:1024800087FD02C081E001C083E08093F4010E94D7
:10249000DD0D8091E10083FF29C08091E20083FF80
:1024A00025C08091E100877F8093E10082E08093E6
:1024B000F4011092F0018091E1008E7F8093E100A1
:1024C0008091E2008E7F8093E2008091E200806143
:1024D0008093E20042E060E080E00E94B4108091CE
:1024E000F00088608093F0000E94D50DFF91EF917D
:1024F000BF91AF919F918F917F916F915F914F911C
:102500003F912F910F900FBE0F901F9018951F9223
:102510000F920FB60F9211242F933F934F935F9317
:102520006F937F938F939F93AF93BF93CF93DF93DB
:10253000EF93FF93C091E900CF708091EC00D82F0A
:10254000D17080FDD0E81092E9008091F000877F83
:102550008093F00078940E94CB121092E900809151
:10256000F00088608093F000CD2BCF70C093E9001D
:10257000FF91EF91DF91CF91BF91AF919F918F919B
:102580007F916F915F914F913F912F910F900FBE6F
:102590000F901F9018951F93CF93DF93CDB7DEB7A1
:1025A000AA970FB6F894DEBF0FBECDBFE5EFF1E0FE
:1025B00088E08E0F9091F10091938E13FBCF0E94D3
:1025C0003D0E8091E80083FF1FC18091F50190913D
:1025D000F601492F50E04A30510508F015C1FA01C3
:1025E000EA5AFF4F0C945229803881F0823809F062
:1025F0000BC18091F9018F708093E9008091EB000D
:1026000085FB882780F91092E90006C08091F101CE
:102610009091F201911182609091E800977F9093E0
:10262000E8008093F1001092F100C8C0282F2D7FA0
:1026300009F0EAC0882319F0823061F0E5C080918A
:10264000F701813009F0E0C0933009F080E0809319
:10265000F2012BC08091F701811127C08091F9010F
:102660008F7009F4D1C08093E9002091EB0020FF26
:102670001CC0933021F48091EB00806214C09091D3
:10268000EB0090619093EB0021E030E0A90102C0E3
:10269000440F551F8A95E2F74093EA001092EA0032
:1026A0008091EB0088608093EB001092E9008091AC
:1026B000E800877F86C08111A7C01091F7011F77BE
:1026C0008091E3008078812B8093E3008091E80083
:1026D000877F8093E8000E94E9108091E80080FFE6
:1026E000FCCF8091E30080688093E300111102C069
:1026F00082E001C083E08093F40186C0805882307C
:1027000008F082C08091F7019091F8018C3D53E070
:10271000950779F583E08A838AE289834FB7F89435
:10272000DE01139620E03EE051E2E32FF0E050930B
:102730005700E49120FF03C0E295EF703F5FEF7018
:102740008E2F90E0EA3010F0C79601C0C0968D93AE
:102750009D932F5F243149F74FBF8091E800877F19
:102760008093E8006AE270E0CE0101960E94F00FCB
:1027700014C0AE014F5F5F4F6091F9010E94370FA7
:10278000BC01009709F440C09091E800977F9093B6
:10279000E80089819A810E9453108091E8008B772C
:1027A0008093E80031C0803879F58091E800877F18
:1027B0008093E8008091F0018093F1008091E8001F
:1027C0008E778093E8000E94E9101EC081111CC022
:1027D0009091F7019230C0F48091E800877F809358
:1027E000E8009093F0010E94E9108091F0018111BE
:1027F00006C08091E30087FD02C081E001C084E053
:102800008093F4010E94240E8091E80083FF0AC0A7
:102810008091E800877F8093E8008091EB008062E0
:102820008093EB00AA960FB6F894DEBF0FBECDBF23
:10283000DF91CF911F910895CF938091F401882368
:10284000A1F0C091E900CF709091EC00892F8170C8
:1028500090FD80E8C82B1092E9008091E80083FD8C
:102860000E94CB12CF70C093E900CF91089590934E
:10287000800180937F010895E0917F01F0918001B4
:10288000309721F00190F081E02D099480E00895C7
:10289000EF92FF920F931F93CF93DF93E0917F010D
:1028A000F09180013097B1F18C010280F381E02D2D
:1028B00009958091DF0182FF2DC080FF04C084E470
:1028C00095E00E94C406E80110E18EE3E82E85E061
:1028D000F82E8091DF0180FF0BC088811F928F93BB
:1028E000FF92EF920E945D070F900F900F900F9054
:1028F000115021961111EDCF8091DF0180FF0AC0A8
:102900008CE395E0DF91CF911F910F91FF90EF90B5
:102910000C94C406DF91CF911F910F91FF90EF901F
:102920000895E0917F01F0918001309721F00480BB
:10293000F581E02D0994089520917D0130917E016B
:102940008217930771F090937E0180937D01E0914F
:102950007F01F0918001309721F00680F781E02D12
:102960000994089520917B0130917C01821793078F
:1029700071F090937C0180937B01E0917F01F09155
:102980008001309721F00084F185E02D09940895AD
:1029900008950C94C8140E9491200E944A0B0C9434
:1029A0001721CF93DF931F92CDB7DEB79091DF0150
:1029B00092FF10C090FF0EC01F928F9326E535E066
:1029C0003F932F9389830E945D070F900F900F9084
:1029D0000F9089810F90DF91CF910C94340B5F920F
:1029E0006F927F928F929F92AF92BF92CF92DF921F
:1029F000EF92FF920F931F93CF93DF9300D000D0FD
:102A00001F92CDB7DEB70E948F0B9AE8C92E91E0D6
:102A1000D92E03E010E0AA24A394B12C502E802FCD
:102A20000E94200C4C01F601729062906F016826A2
:102A3000792661147104A1F40150110978F78FEF20
:102A400089838A831B820E949A208160782F9D83CC
:102A50008C8349815A816B818D810E949F1538C07A
:102A60008091DF0181FD0E94290C2AE030E0750190
:102A7000022E02C0EE0CFF1C0A94E2F7C701862169
:102A80009721892B09F129835A828E209F2091E07A
:102A9000892809F490E09B830E949A208160782F16
:102AA0009D838C8349815A816B818D810E949F1502
:102AB000000F111FF801EE57FE4F80819181E8262B
:102AC000F926F182E08204C02150310980F6B4CFAA
:102AD0000E946423109181010E943C141817D1F0C8
:102AE0000E943C14809381010F900F900F900F90E3
:102AF0000F90DF91CF911F910F91FF90EF90DF909A
:102B0000CF90BF90AF909F908F907F906F905F908D
:102B10000C94D1140F900F900F900F900F90DF91A5
:102B2000CF911F910F91FF90EF90DF90CF90BF90CA
:102B3000AF909F908F907F906F905F900895CF930C
:102B4000DF93CDB7DEB72B970FB6F894DEBF0FBE7D
:102B5000CDBF4F83588769877A878B87DE011196AF
:102B600086E0FD0111928A95E9F785E0FE0137962E
:102B700001900D928A95E1F749815A816B817C81A0
:102B80008D819E810E94F01B2B960FB6F894DEBFBC
:102B90000FBECDBFDF91CF910895CF93882309F465
:102BA000C2C0C82F823859F40E943C1481FDBBC0BA
:102BB00089E30E94CA1E0E94B91F89E30CC08338B2
:102BC00079F40E943C1480FDAEC083E50E94CA1EC9
:102BD0000E94B91F83E50E941D1FCF910C94B91F5D
:102BE000843859F40E943C1482FD9DC087E40E9401
:102BF000CA1E0E94B91F87E4EECF8CEF8C0F813A7A
:102C000048F48C2F0E94BB2681118DC08C2F0E940E
:102C1000CA1EE3CF80E28C0F883048F4C77081E091
:102C200001C0880FCA95EAF70E94721FD6CF8BE5C4
:102C30008C0F833078F4C53A29F0C63A31F083E836
:102C400090E005C081E890E002C082E890E0CF917A
:102C50000C949C1488E58C0F833108F064C0C83A4A
:102C600039F1C93A41F1CA3A49F1CB3A51F1CC3A7A
:102C700059F1CD3A61F1C03B69F1CE3A71F1CF3AE9
:102C800079F1C13B81F1C23B89F1C33B91F1C43B76
:102C900099F1C53BA1F1C63BA9F1C73BB1F1C83BD6
:102CA000B9F1C93BC1F1CA3BC9F180E090E038C03D
:102CB00082EE90E035C089EE90E032C08AEE90E07E
:102CC0002FC085EB90E02CC086EB90E029C087EB0D
:102CD00090E026C08CEC90E023C08DEC90E020C00A
:102CE00083E891E01DC08AE891E01AC082E991E092
:102CF00017C084E991E014C081E292E011C083E240
:102D000092E00EC084E292E00BC085E292E008C03F
:102D100086E292E005C087E292E002C08AE292E099
:102D2000CF910C94B214CF910895882309F44BC02D
:102D3000823859F40E943C1481FF45C089E30E9407
:102D4000CA1E0E94B91F89E30CC0833871F40E9427
:102D50003C1480FF38C083E50E94CA1E0E94B91F40
:102D600083E50E941D1F0C94B91F843859F40E94FA
:102D70003C1482FF28C087E40E94CA1E0E94B91F2B
:102D800087E4EFCF9CEF980F913A58F390E2980FB9
:102D9000983050F4877091E001C0990F8A95EAF756
:102DA000892F0E94781FDFCF9BE5980F933020F486
:102DB00080E090E00C949C14885A833120F480E0E9
:102DC00090E00C94B2140895882321F00E94721FA1
:102DD0000C94B91F0895882321F00E94781F0C9449
:102DE000B91F08957F928F929F92AF92BF92CF9218
:102DF000DF92EF92FF920F931F93CF93DF931F9277
:102E0000CDB7DEB77C01C62E772EFC010581029579
:102E10000F70128111110E948F1F0E94C31E882300
:102E200079F0112369F080E28C0D883048F082E05F
:102E30000E94AC1E0E94C31E91E0D82ED92601C06C
:102E4000D12CE72DE295EF70F0E0E05AFF4F0C94A3
:102E50005229872D807F072D0F70882311F002954E
:102E6000007F112389F0002309F498C180E28C0DC2
:102E7000883020F4802F0E94721F03C0802F0E9490
:102E8000821F0E94B91F8AC18C2D0E9495160023B3
:102E900009F49DC180E28C0D883020F4802F0E94BF
:102EA000781F03C0802F0E94881F0E94B91F8FC106
:102EB000872D807F972D9F70803211F4892F03C05A
:102EC000892F8295807FCC2021F0F1E0CF16A1F0F0
:102ED0001DC0112339F0002319F1013009F50E94BA
:102EE000A21F75C1002319F0013009F470C1898354
:102EF0000E94A51F898110C1112321F0063008F01E
:102F000066C10EC0053008F062C106C1112359F038
:102F1000002331F0F701958190FF40C19F709583A8
:102F20000E94E41654C1002309F4F6C03DC1872D68
:102F300086958695837090E0009719F0019761F06F
:102F400046C1112321F08C2D972D937002C080E093
:102F500090E00E949C143BC1112321F08C2D972DF1
:102F6000937002C080E090E00E94B21430C18C2DBA
:102F7000112319F00E94EA2102C00E9452220E94ED
:102F8000D72225C1872D837009F052C011111FC1AE
:102F90008C2D829586958770880F880F9C2D9F7049
:102FA000892E912CA12CB12C082E04C0880C991CC0
:102FB000AA1CBB1C0A94D2F7C4FE14C00FE010E098
:102FC00020E030E0B901A80104C0440F551F661F7E
:102FD000771F8A95D2F7CB01BA01609570958095DD
:102FE000909503C060E070E0CB01272D26952695D3
:102FF000237030E02230310569F02330310589F04B
:10300000682979298A299B292130310571F00E948C
:10301000381DDDC0682979298A299B290E94541D01
:10302000D6C00E94381DC501B4010E941C1DCFC02E
:10303000112319F0872D817001C08695882309F42A
:10304000C6C08C2D829586958770880F880F9C2D21
:103050009F70892E912CA12CB12C082E04C0880CB5
:10306000991CAA1CBB1C0A94D2F7C4FE14C00FE022
:1030700010E020E030E0B901A80104C0440F551F62
:10308000661F771F8A95D2F7CB01BA0160957095BC
:103090008095909503C060E070E0CB01272D2695C8
:1030A00026952370422F50E04230510569F043309D
:1030B000510589F0682979298A299B2941305105D0
:1030C00071F00E94121E83C0682979298A299B29E0
:1030D0000E942E1E7CC00E94121EC501B4010E94D7
:1030E000F61D75C08C2D90E0FC01E05EF109E53124
:1030F000F10508F04FC0E059FF4F0C9452290C2DF8
:103100000F70872D8F71112321F00E948F1D802F4A
:1031100007CF0E94B01D802F0E94EB1658C01123CC
:1031200041F0053008F053C0872D8F710E94D51DE6
:103130004EC0063008F04BC0F7CF112339F0872D71
:103140008F710E948F1D43C01123C9F3872D8F718A
:103150000E94B01D3CC0112329F0872D8F710E9461
:103160007A1D35C00E94701D32C0112351F0172DF9
:103170001F71812F0E948F1D63E0812F0E94A31E6B
:1031800026C081E00E94AC1E023008F182E00E945D
:10319000AC1E1DC0112331F0002389F28C2D0E943A
:1031A000CD1515C0002391F28C2D0E9495160FC0ED
:1031B000472D4F706C2DC7010E9476070E94941C0A
:1031C00006C0472D4F706C2DC7010E943908DD20C5
:1031D000F9F00E949F1E80FD1BC0F70112820E9421
:1031E000991E0E948F1DC7010E9417190E94991EE7
:1031F0000F90DF91CF911F910F91FF90EF90DF9093
:10320000CF90BF90AF909F908F907F900C94B01D07
:103210000F90DF91CF911F910F91FF90EF90DF9072
:10322000CF90BF90AF909F908F907F9008950F9315
:103230001F93CF93DF93EC01888199812B813C818F
:10324000232BB9F09F3F11F48F3F99F0CE010E94DC
:103250008D07882371F0688179818A810E94951E8B
:103260008C010E944A1E0E94111DB801CE010E94CD
:10327000F216DF91CF911F910F9108950E948F1F39
:103280000E949F1F0E94641F0E94B91F0E940A246F
:103290000E94D72280E090E00E949C1480E090E0A1
:1032A0000C94B2140E947F1F0C943E190E948A1E37
:1032B000292F22952F7030E02C3031054CF42A3024
:1032C00031056CF42250310922303105A8F407C0D1
:1032D0002C30310569F02F30310551F00DC0803FA1
:1032E00069F018F4803E40F409C0843F29F406C018
:1032F00093FB882780F9089580E0089581E0089580
:10330000CF93DF9300D000D01F92CDB7DEB70F90E0
:103310000F900F900F900F90DF91CF910895CF9362
:10332000DF9300D000D000D0CDB7DEB726960FB621
:10333000F894DEBF0FBECDBFDF91CF9108951F93EC
:10334000CF93DF93C0918A0116E080918B01C8175B
:1033500099F0D0E01C9FF0011D9FF00D1124E4575F
:10336000FE4F4081518162817381848195810E94E9
:103370008F192196C770E9CFDF91CF911F910895E2
:103380004091BC015091BD016091BE017091BF019F
:103390008091C0019091C1010C948F198091C1015D
:1033A00082958F7009F054C08091BE01882309F482
:1033B0004FC080918A01A0918B016091BC017091F6
:1033C000BD014091BF015091C001B6E08A1709F4D8
:1033D0003FC090E041155105C1F17F3F11F46F3FAF
:1033E000A1F1B89FF001B99FF00D1124E457FE4FF1
:1033F000218172132AC02081621327C022812111EA
:1034000024C0238134812417350710F42150310959
:10341000241B350B283C3105C0F42091C1012F70CD
:1034200020612093C10126E0289FF001299FF00D23
:103430001124EF56FE4F80818F70806180838CEB6A
:1034400091E00E9417190C949F1901968770BECFC6
:103450000895CF92DF92EF92FF920F931F93CF9335
:10346000DF93CDB7DEB762970FB6F894DEBF0FBE1D
:10347000CDBF8C0185E0F801DE011D9601900D9213
:103480008A95E1F7D8014C9111965C9111971296AB
:103490006C9112971396CD90DC9014973091BC01EB
:1034A0007091BD018091BF019091C001009709F416
:1034B0006BC17F3F19F43F3F09F466C1E090BE0144
:1034C000EE2009F4C0C02091C101C816D90628F029
:1034D000F601E81BF90BCF0104C0809590958C0D87
:1034E0009D1DFF24F394883C910578F0F12C207FFA
:1034F00009F0C6C07C2DD98AC88A89890E948019A2
:103500008CEB91E00E941719B1C0822F807F09F0E7
:1035100046C0751314C0341312C0611110C02F704F
:1035200020612093C1010E94C0198CEB91E00E94A0
:1035300017198091C101D80115968C932EC0CD2802
:1035400019F15F3F11F44F3FF9F0F62E61111CC0E5
:1035500080918A0120918B0136E0821709F45AC0CC
:1035600090E0389FF001399FF00D1124E457FE4F91
:103570007181571306C07081471303C072817111A6
:1035800003C001968770E9CFF62E662309F418C1AF
:103590008091C10181608093C101F12C11C175132B
:1035A00008C0341306C0611104C08091C101D80164
:1035B000C3C04D875E878D859E856A8B0E94561994
:1035C0006A898823E1F16623D1F12091C101822F1C
:1035D00082958F7090E0029774F08091BC01909179
:1035E000BD0198878F831986DB86CA862C87CE011A
:1035F00007960E94171986E0F801ACEBB1E0019044
:103600000D928A95E1F70E94CE190E94C019FF24FD
:10361000F394D6C04D875E878D859E850E948A1E55
:10362000292F22952F7030E0223031050CF0BCC0DC
:103630009F7009F0B6C0805E883008F4C1C0C80130
:103640000E941719E4CFC816D90608F453C0F60132
:10365000E81BF90BCF01883C910508F450C0F12C10
:103660007C2DD98AC88A89890E948019ECEBF1E007
:1036700086E0DF011D928A95E9F70E94C019A0C07B
:10368000751314C0341312C0611110C08091C101B0
:10369000F8018583C8010E94171986E0ECEBF1E080
:1036A000DF011D928A95E9F7FE2C8AC04D875E875F
:1036B0008D859E856A8B0E9456196A89882309F434
:1036C000BECF662309F4BBCF2091C101822F829522
:1036D0008F7090E002970CF48ECF8091BC01909196
:1036E000BD019A8389831B82DD82CC822E83CE0129
:1036F00001967FCF809590958C0D9D1DACCFF62EB9
:10370000662309F49CCF75132EC034132CC020916E
:10371000C10120FD1FC0822F82958F70D9F0D80182
:1037200015962C9315978F3049F08F5F982F9295AF
:10373000907F822F8F70892B15968C93C8010E94E1
:10374000171986E0F801ACEBB1E001900D928A9573
:10375000E1F793CF86E0F801ACEBB1E001900D9278
:103760008A95E1F72DC04D875E878D859E850E94E5
:103770005619811140CF8091C10181608093C101B0
:10378000C8010E9417191CC0662309F458CF4D8741
:103790005E878D859E850E945619882309F44FCF38
:1037A0002ACF811148CF0CC0243031050CF047CF0F
:1037B0009F7009F440CFF8019581907F09F03BCFCD
:1037C0008F2D62960FB6F894DEBF0FBECDBFDF918E
:1037D000CF911F910F91FF90EF90DF90CF900895C0
:1037E0001F93CF93DF93CDB7DEB72C970FB6F89426
:1037F000DEBF0FBECDBF4F83588769877A878B871F
:103800009C87CE0107960E94291A882369F08F8130
:1038100098852A853B85232BF1F19F3F09F063C0F2
:103820008F3F09F060C037C086E0FE013796DE01A9
:10383000119601900D928A95E1F76F817885EA855E
:10384000FB85309741F17F3F11F46F3F21F12091CB
:103850008B0130E0C90101968770992740918A0158
:1038600050E08417950709F447C069837A83FD8384
:10387000EC8396E0929FD001939FB00D1124A45742
:10388000BE4FFE01319601900D929A95E1F780931B
:103890008B010E949F1916E080918A0190918B0103
:1038A0008917C1F1189FC001112484579E4F0E94AF
:1038B000291A882379F1E0918A011E9FF0011124D1
:1038C000E457FE4F408151816281738184819581EB
:1038D0000E948F1980918A0190E001968770992744
:1038E00080938A01D9CF4F81588569857A858B85E8
:1038F0009C850E948F19CFCF0E94521910928B0184
:1039000010928A01ECEBF1E086E0DF011D928A95CE
:10391000E9F7C1CF2C960FB6F894DEBF0FBECDBF2E
:10392000DF91CF911F910895EF92FF920F931F9314
:10393000CF93DF938C01009709F46CC0F12CEE2437
:10394000E394E8012196F8018491843740F48430AF
:1039500008F051C0813081F0823019F15BC08537A9
:1039600009F444C0A8F19CE7980F903708F052C0C2
:103970008F770E94951641C00E5F1F4FFE01C491C4
:1039800080E28C0F883048F4C7708E2D01C0880FFC
:10399000CA95EAF70E94921F14C08C2F0E94CD1581
:1039A0002DC00E5F1F4FFE01C49180E28C0F883046
:1039B00058F4C7708E2D01C0880FCA95EAF70E948F
:1039C000981F0E94B91F1AC08C2F0E94951616C00E
:1039D0000E5F1F4FFE01C491CC2381F08FE99FE061
:1039E0000197F1F700C00000C150F6CF0E5F1F4FE6
:1039F000FE01F49003C00E94CD158E018F2D882307
:103A000009F49FCFEFE9FFE03197F1F700C0000024
:103A10008150F5CFDF91CF911F910F91FF90EF90E3
:103A2000089508956093C6017093C7018093C801FB
:103A30009093C9010C943E190F931F930091C601F6
:103A40001091C7012091C8013091C901DC01CB015F
:103A5000802B912BA22BB32B8093C6019093C7018F
:103A6000A093C801B093C9011F910F910C943E1906
:103A70000F931F930091C6011091C7012091C801B7
:103A80003091C901DC01CB0180239123A223B32310
:103A90008093C6019093C701A093C801B093C90158
:103AA0001F910F910C943E190F931F930091C60123
:103AB0001091C7012091C8013091C901DC01CB01EF
:103AC00080279127A227B3278093C6019093C7012F
:103AD000A093C801B093C9011F910F910C943E1996
:103AE0001092C2011092C3011092C4011092C5013C
:103AF0000C943E1941E050E060E070E004C0440FD7
:103B0000551F661F771F8A95D2F74093C2015093C5
:103B1000C3016093C4017093C5010C943E1941E048
:103B200050E060E070E004C0440F551F661F771F2F
:103B30008A95D2F78091C2019091C301A091C401EE
:103B4000B091C501482B592B6A2B7B2B4093C201A6
:103B50005093C3016093C4017093C5010C943E1946
:103B600041E050E060E070E004C0440F551F661F64
:103B7000771F8A95D2F74095509560957095809102
:103B8000C2019091C301A091C401B091C501482325
:103B900059236A237B234093C2015093C30160934E
:103BA000C4017093C5010C943E1941E050E060E0FF
:103BB00070E004C0440F551F661F771F8A95D2F727
:103BC0008091C2019091C301A091C401B091C5013F
:103BD000482759276A277B274093C2015093C30186
:103BE0006093C4017093C5010C943E190F931F9309
:103BF0000091C2011091C3012091C4013091C5010F
:103C0000DC01CB01802B912BA22BB32B8093C20123
:103C10009093C301A093C401B093C5011F910F916C
:103C20000C943E190F931F930091C2011091C30190
:103C30002091C4013091C501DC01CB018023912387
:103C4000A223B3238093C2019093C301A093C40124
:103C5000B093C5011F910F910C943E190F931F93C0
:103C60000091C2011091C3012091C4013091C5019E
:103C7000DC01CB0180279127A227B3278093C201C3
:103C80009093C301A093C401B093C5011F910F91FC
:103C90000C943E190895CF92DF92EF92FF920F930A
:103CA0001F93CF93DF938C01C090C601D090C701C2
:103CB000E090C801F090C9018091C2019091C301C8
:103CC000A091C401B091C501C82AD92AEA2AFB2AC9
:103CD000CFE1D0E0D701C6010C2E04C0B695A79560
:103CE000979587950A94D2F780FF06C0B8018C2F6C
:103CF0000E94990A019721F4219760F780E001C0A2
:103D00008C2FDF91CF911F910F91FF90EF90DF905B
:103D1000CF900895CF93DF93EC010E944B1EBE011C
:103D20000E94990ADF91CF910895CB010E948A1ECB
:103D300008958091CA01859585958595089580910E
:103D4000CA018770089598E0899F90011124262B5D
:103D50002093CA010C948F1D2091CA018095822363
:103D60008093CA01982F977069F430E0482F552747
:103D700047FD50952417350729F08595859585953C
:103D80000C94B01D08959091CA01977081E009F4D8
:103D900080E0089590910B01992321F090910C01FE
:103DA000911109C020910D0130910E01F901329657
:103DB0009FEF40E030C0982F9695969596959F304E
:103DC000A0F4E0910D01F0910E01E90FF11D877053
:103DD00021E030E0A90102C0440F551F8A95E2F7A7
:103DE000CA019181892B818308959091DF0190FF11
:103DF00023C01F928F938DE895E09F938F930E942D
:103E00005D070F900F900F900F9008959F3F39F02E
:103E10004F5F4E3041F051915813F8CF0DC0511102
:103E2000F7CF942FF5CF9F3F39F0F901E90FF11D3E
:103E300097FDFA9582830895089590910B01992337
:103E400021F090910C01911109C020910D01309148
:103E50000E01F9013296205F3F4F30C0982F9695A2
:103E6000969596959F30A8F4E0910D01F0910E0182
:103E7000E90FF11D877021E030E0A90102C0440F75
:103E8000551F8A95E2F7CA01809591818923818324
:103E900008959091DF0190FF16C01F928F938FE6D7
:103EA00095E09F938F930E945D070F900F900F9066
:103EB0000F9008953196E217F30729F09081981337
:103EC000F9CF1082F7CF089581E090E0E0910D01E5
:103ED000F0910E01E80FF91F1082019680319105D3
:103EE000A9F708959091DE01892B8093DE01089552
:103EF00080959091DE0189238093DE0108951092D0
:103F0000DE0108959091DD01892B8093DD010895F4
:103F100080959091DD0189238093DD0108951092B1
:103F2000DD0108959091DC01892B8093DC010895D7
:103F300080959091DC0189238093DC010895109293
:103F4000DC0108958093CB0108951092CB01089570
:103F500080910D0190910E01FC0131969C01205F32
:103F60003F4F80E0919191118F5FE217F307D1F7F6
:103F70000895E0910D01F0910E018091DE018083A2
:103F8000E0910D01F0910E0190818091DD01892B6E
:103F90008083E0910D01F0910E0190818091DC0110
:103FA000892B80838091CB01882361F0E0910D0102
:103FB000F0910E019081892B80830E94A81F8111AE
:103FC0001092CB0180910D0190910E010C94481438
:103FD0009093490180934801089520E0009739F0BB
:103FE000AC0141505109842395232F5FF7CF822FD5
:103FF00008958295982F9C7C392F36953695282FD9
:10400000237344E0249FC0011124932F982B292F60
:104010002A7A2695892F8575880F822B08951F93FC
:10402000CF93DF931F92CDB7DEB799830E94F91F1C
:10403000182F9981892F0E94F91F212F30E0322FEC
:104040002227A901482BCA010F90DF91CF911F9120
:1040500008958091F401843021F11092E00120E470
:1040600088E190E00FB6F894A895809360000FBEA9
:104070002093600080E00E94340B83B7817F8460CE
:1040800083BF83B7816083BF7894889583B78E7F21
:1040900083BF88E10FB6F8948093600010926000AF
:1040A0000FBE0895089508950E9452200E948F0B1C
:1040B0000E9453200E94630C91E0811101C090E0A6
:1040C000892F08950E9452190E943C140C94340BBD
:1040D0001F920F920FB60F9211248F939F93AF935D
:1040E000BF938091E001811113C08091E101909113
:1040F000E201A091E301B091E4014196A11DB11D3F
:104100008093E1019093E201A093E301B093E40175
:10411000BF91AF919F918F910F900FBE0F901F9005
:10412000189582E084BD93E095BD9AEF97BD80938A
:104130006E0008952FB7F8948091E1019091E2010B
:10414000A091E301B091E4012FBF0895CF92DF92D7
:10415000EF92FF920F931F932FB7F8944091E101D4
:104160005091E2016091E3017091E4012FBF6A0177
:104170007B01EE24FF248C0120E030E0C016D10644
:10418000E206F30610F4415051099A01281B390B3D
:10419000C9011F910F91FF90EF90DF90CF9008958C
:1041A0001F920F920FB60F9211248F939F93AF938C
:1041B000BF938091E1019091E201A091E301B09160
:1041C000E4010196A11DB11D8093E1019093E201EC
:1041D000A093E301B093E401BF91AF919F918F91C0
:1041E0000F900FBE0F901F9018950E943A11F894EF
:1041F0002FEF87EA91E6215080409040E1F700C020
:10420000000087E090EBDC018093FE019093FF01BA
:10421000A0930002B09301029CE088E10FB6F894ED
:10422000A895809360000FBE90936000FFCF0E941E
:104230004C21811102C00E9432210E94572180939B
:10424000DF010E945F218093FD0187FB882780F9B1
:1042500080930C010E945B21682F70E080E090E069
:104260000C94121D6DEE7EEF80E090E00E948C2990
:1042700060E082E090E00E947A2960E083E090E0D4
:104280000E947A2960E084E090E00E947A2960E050
:1042900085E090E00C947A2980E090E00E947429F7
:1042A00021E08D3E9E4F09F020E0822F089582E0AC
:1042B00090E00C946C2983E090E00C946C2984E0ED
:1042C00090E00C946C29682F84E090E00C947A299B
:1042D0008091E70180FF0BC06091120185E0689F2B
:1042E000B001112475956795759567952BC081FF71
:1042F00009C06091120185E0689FB0011124759595
:10430000679520C082FF07C06091120185E0689F19
:10431000B001112417C09091E8019923D1F0609168
:104320001101961788F72091120185E0289F9001CE
:104330001124929FA001939F500D112470E0CA0197
:104340000E943E296038710540F46115710539F00D
:1043500002C065E070E0862F08958FE7089581E040
:1043600008958091E70180FF08C06091100170E01E
:10437000759567957595679521C081FF06C0609119
:10438000100170E07595679519C082FF04C06091B7
:10439000100170E010C09091E8019923C1F0609184
:1043A0000F019617A0F780911001899FC001112479
:1043B00070E00E943E296038710528F4611571058E
:1043C00021F0862F08958FE7089581E0089561E038
:1043D00070E0F4CF803F21F40E946821819504C0F1
:1043E000813F29F40E9468218093EB010895823F68
:1043F00021F40E946821819504C0833F29F40E9422
:1044000068218093EA010895893F19F40E94B1213F
:1044100005C08A3F31F40E94B12181958093EC015F
:1044200008958B3F21F40E94B121819504C08C3FF7
:1044300029F40E94B1218093ED010895843F21F475
:104440008091E901816017C0853F21F48091E901E5
:10445000826011C0863F21F48091E90184600BC025
:10446000873F21F48091E901886005C0883F31F4DD
:104470008091E90180618093E90108958D3F21F4E5
:104480008091E70181600BC08E3F21F48091E701AC
:10449000826005C08F3F29F48091E701846080939A
:1044A000E7010895803F39F48091EB0187FF6CC0EC
:1044B0001092EB0169C0813F29F48091EB0118163D
:1044C000BCF362C09091EA01823F29F497FF5CC07F
:1044D0001092EA0159C0833F19F41916CCF354C065
:1044E000893F41F48091EC0118160CF04DC01092F8
:1044F000EC014AC08A3F29F48091EC0187FF44C057
:10450000F6CF8B3F39F48091ED0187FF3DC01092CB
:10451000ED013AC08C3F29F48091ED011816BCF3EF
:1045200033C0843F21F48091E9018E7F17C0853F1D
:1045300021F48091E9018D7F11C0863F21F48091A3
:10454000E9018B7F0BC0873F21F48091E901877FD0
:1045500005C0883F31F48091E9018F7E8093E901A5
:1045600013C08D3F21F48091E7018E7F0BC08E3FF9
:1045700021F48091E7018D7F05C08F3F29F4809160
:10458000E7018B7F8093E7018091EA0181110EC0E2
:104590008091EB0181110AC08091EC01811106C06C
:1045A0008091ED01811102C01092E801089580917F
:1045B000DF0183FF7EC082ED95E00E94C4068091FA
:1045C000E9011F928F938DEC95E09F938F930E944A
:1045D0005D078BEC95E00E94C4068091EA01282FCC
:1045E000332727FD30953F938F9388EC95E09F9379
:1045F0008F930E945D0786EC95E00E94C40680912F
:10460000EB01282F332727FD30953F938F9383ECC1
:1046100095E09F938F930E945D0781EC95E00E9447
:10462000C4068091EC01282F332727FD30953F9356
:104630008F938EEB95E09F938F930E945D078CEB99
:1046400095E00E94C4068091ED01282F332727FDB5
:1046500030953F938F9389EB95E09F938F930E94C2
:104660005D0786EB95E00E94C4068091E8011F92E9
:104670008F9383EB95E09F938F930E945D0781EB6F
:1046800095E00E94C4068091E7011F928F938EEA05
:1046900095E09F938F930E945D078BEA95E00E94BF
:1046A000C4068DB79EB74C960FB6F8949EBF0FBE4A
:1046B0008DBF89EE91E00E9491140E949A20909300
:1046C000E6018093E50108951F93CF93DF938091D6
:1046D000E5019091E6010E94A620AC019091E801CD
:1046E000992321F02091130130E006C0209114019C
:1046F0008AE0289F900111244217530708F486C0CE
:104700008091EA01C091EB01D091EC011091ED0193
:10471000811107C0C11176C0D11174C0111172C0CE
:1047200075C09F3F19F09F5F9093E801181624F41D
:104730000E9468218093EA018091EA0187FF05C009
:104740000E94682181958093EA011C1624F40E943E
:1047500068218093EB018091EB0187FF05C00E94E7
:10476000682181958093EB016091EA01662339F11C
:10477000C091EB01CC2319F1772767FD7095872F46
:10478000972F0E94432823E333E343E35FE30E9430
:10479000A7280E9410286093EA016C2F772767FDF5
:1047A0007095872F972F0E94432823E333E343E339
:1047B0005FE30E94A7280E9410286093EB011D165A
:1047C00024F40E94B1218093EC018091EC0187FFD9
:1047D00005C00E94B12181958093EC01111624F44B
:1047E0000E94B1218093ED018091ED0187FF05C00A
:1047F0000E94B12181958093ED01DF91CF911F91AE
:104800000C94D7229F3F09F08ECF96CFDF91CF91A6
:104810001F910895E9EEF1E085E0DF011D928A9590
:10482000E9F71092E8011092E701089585EF97E00B
:104830000E94C4061F9281E08F931F9285E08F93A0
:1048400087EA97E09F938F930E945D070F900F90E8
:104850000F900F900F900F9008958330E9F128F496
:10486000813061F0823009F10895853009F462C029
:1048700008F449C0863009F474C008958091140189
:10488000262F30E0280F311D2F3F310524F4680F0B
:104890006093140103C08FEF809314018091140181
:1048A0001F928F9380EE96E072C080911301262FA5
:1048B00030E0280F311D2F3F310524F4680F60933D
:1048C000130103C08FEF80931301809113011F9296
:1048D0008F938EEC96E05BC080911201262F30E022
:1048E000280F311D2F3F310524F4680F609312010A
:1048F00003C08FEF80931201809112011F928F935A
:104900008BEB96E044C080911101262F30E0280FF8
:10491000311D2F3F310524F4680F6093110103C04E
:104920008FEF80931101809111011F928F9386EA7E
:1049300096E02DC080911001262F30E0280F311D08
:104940002F3F310524F4680F6093100103C08FEFEF
:1049500080931001809110011F928F938DE896E053
:1049600016C080910F01262F30E0280F311D2F3FF8
:10497000310524F4680F60930F0103C08FEF80931B
:104980000F0180910F011F928F9382E796E09F9312
:104990008F930E945D070F900F900F900F900895D6
:1049A000833081F128F4813059F08230D1F00895BC
:1049B000853009F449C0B8F1863009F456C008952D
:1049C00080911401681720F4861B8093140102C0A3
:1049D00010921401809114011F928F9383E696E048
:1049E00054C080911301681720F4861B8093130133
:1049F00002C010921301809113011F928F9381E5E1
:104A000096E043C080911201681720F4861B8093C2
:104A1000120102C010921201809112011F928F9315
:104A20008EE396E032C080911101681720F4861B56
:104A30008093110102C010921101809111011F9207
:104A40008F9389E296E021C080911001681720F4CD
:104A5000861B8093100102C01092100180911001FA
:104A60001F928F9380E196E010C080910F0168172C
:104A700020F4861B80930F0102C010920F018091D9
:104A80000F011F928F9385EF95E09F938F930E9464
:104A90005D070F900F900F900F900895CF93C82F40
:104AA0001F928F938AEF98E09F938F930E945D07E8
:104AB00081E090E0A0E0B0E0BC01CD0104C0660F51
:104AC000771F881F991FCA95D2F70E94121D0F9059
:104AD0000F900F900F90CF910C945219CF93873273
:104AE000A8F58E3108F035C1803109F4A5C0F8F47D
:104AF000873009F465C0A8F4863009F030C1809190
:104B0000DF01817F8E7F8093DF018FE79AE00E9433
:104B1000C40680EE9CE00E94C40681E08093EF0111
:104B20004DC08B30F1F18E3009F472C018C186315E
:104B300009F4B6C020F4813109F4F9C010C18931FB
:104B400009F497C08B3109F44FC009C1883349F18A
:104B500050F4893209F4FFC0853309F4FCC0873270
:104B600009F4F9C0FCC0833409F4F5C028F48A3391
:104B700008F4F5C08953F0C0883409F0F0C00E94F1
:104B8000521984EC9CE00E94C4062FEF83ED90E361
:104B9000215080409040E1F700C000000E94F520C5
:104BA0000DC086EA9AE062C08BEA9CE00E94C406CF
:104BB0008091DF01897F877F8093DF01C1E0D4C0CE
:104BC0008091DF01C82FC095C170C0FB80F9809330
:104BD000DF01CC2349F388EB9CE00E94C40680915E
:104BE000DF01866088603DC09091DF0191FBCC279A
:104BF000C0F981E0C827892FC0FB81F98093DF01CC
:104C0000CC2319F08EE99CE027C080E99CE02EC0FF
:104C10009091DF0192FBCC27C0F981E0C827892F52
:104C2000C0FB82F98093DF01CC2319F081E89CE07E
:104C300013C081E79CE01AC09091DF0193FBCC2761
:104C4000C0F981E0C827892FC0FB83F98093DF0179
:104C5000CC2351F085E69CE00E94C4068091DF01E0
:104C600081608093DF0180C088E59CE00E94C406DB
:104C7000A5CF80E79AE00E94C40685E49AE00E94EE
:104C8000C4068BE09AE00E94C4068EED99E00E9473
:104C9000C40683EA99E00E94C40688E799E0E6CF5B
:104CA0008AE699E00E94C4060E943C141F928F93EA
:104CB00080E599E09F938F930E945D0780910B019F
:104CC0001F928F9389E399E09F938F930E945D07D2
:104CD00080917A011F928F9386E299E09F938F9340
:104CE0000E945D0780910C011F928F9383E199E0F0
:104CF0009F938F930E945D078091E1019091E20163
:104D0000A091E301B091E401BF93AF939F938F9380
:104D10008FEF98E09F938F930E945D078DB79EB7AA
:104D200046960FB6F8949EBF0FBE8DBF47CF0E9428
:104D30005219C0910C0181E0C827C0930C01CC230B
:104D400029F08EE49CE00E94C4060EC083E49CE03F
:104D50008DCF8D5101C080E00E944E252FCF81E480
:104D60009CE00E94C406C0E08C2FCF91089580E0A3
:104D7000089580E00895CF93C82F8091EF0181308E
:104D800071F020F0823009F44BC042C1E0910D0176
:104D9000F0910E018081823209F03CC107C0E091A0
:104DA0000D01F0910E018081823261F48C2F0E94FE
:104DB000B726811104C08C2F0E946E252FC081E080
:104DC00090E02CC08C2F0E94B926811126C0C431DE
:104DD000E1F070F4CB3081F0C031D1F40E941624A0
:104DE00082EF98E00E94C40682E08093EF0115C034
:104DF000C93259F0C83361F48FE79AE00E94C406C3
:104E000086EF98E00E94C40608C01092EF0104C12A
:104E100080EF98E00E94C406FFC081E08170FEC070
:104E2000C43228F5CE3108F0C1C0CB30A1F1D0F4A6
:104E3000C73009F0D3C08EE18093140182E38093E0
:104E400013018AE08093120184E18093110188E0CC
:104E50008093100188E280930F0186E997E00E9419
:104E6000C406BFC0C33149F1C431C1F0B7C0CB34AF
:104E700009F4A9C028F4C93289F0C83361F0AEC082
:104E8000C13509F49EC0C23509F499C0CE3409F089
:104E9000A5C06AE09EC00E941624A3C08091EE01C6
:104EA000882319F01092EE019CC083EA97E00E94DB
:104EB000C40681E08093EF01B1C08DE797E00E94C6
:104EC000C4068BE697E00E94C406809114011F92ED
:104ED0008F9388E697E09F938F930E945D0786E605
:104EE00097E00E94C40684E597E00E94C406809182
:104EF00013011F928F9381E597E09F938F930E94F8
:104F00005D078FE497E00E94C40680E497E00E946A
:104F1000C406809112011F928F938DE397E09F93B7
:104F20008F930E945D078BE397E00E94C4068AE29C
:104F300097E00E94C406809111011F928F9387E22F
:104F400097E09F938F930E945D0785E297E00E9410
:104F5000C40680E197E00E94C406809110011F9270
:104F60008F938DE097E09F938F930E945D078BE076
:104F700097E00E94C40684EF96E00E94C4068091E8
:104F80000F011F928F9381EF96E09F938F930E9462
:104F90005D078FEE96E00E94C4068DB79EB74896D7
:104FA0000FB6F8949EBF0FBE8DBF1BC0CE51EC2F25
:104FB000F0E0E35CFE4F80818093EE0112C061E07F
:104FC00003C061E006C06AE08091EE010E942D24DA
:104FD00008C08091EE010E94D02403C084E997E0CC
:104FE00013C08091EE01882369F01F928F938EE8A1
:104FF00097E09F938F930E945D070F900F900F9003
:105000000F9004C08BE897E00E94C40681E006C0C0
:105010001092EF0180E002C080E000CFCF910895B0
:1050200004D06894B1118DC0089570D088F09F5756
:1050300090F0B92F9927B751A0F0D1F0660F771FE4
:10504000881F991F1AF0BA95C9F712C0B13081F0C4
:1050500077D0B1E0089574C0672F782F8827B85FA4
:1050600039F0B93FCCF3869577956795B395D9F725
:105070003EF490958095709561957F4F8F4F9F4F2F
:105080000895E89409C097FB3EF49095809570953B
:1050900061957F4F8F4F9F4F9923A9F0F92F96E984
:1050A000BB279395F695879577956795B795F111F9
:1050B000F8CFFAF4BB0F11F460FF1BC06F5F7F4F96
:1050C0008F4F9F4F16C0882311F096E911C07723A8
:1050D00021F09EE8872F762F05C0662371F096E8B1
:1050E000862F70E060E02AF09A95660F771F881F80
:1050F000DAF7880F9695879597F9089557FD905898
:10510000440F551F59F05F3F71F04795880F97FB8B
:10511000991F61F09F3F79F0879508951216130645
:105120001406551FF2CF4695F1DF08C01616170674
:105130001806991FF1CF86957105610508940895A9
:10514000E894BB2766277727CB0197F908950BD002
:1051500078C069D028F06ED018F0952309F05AC0B5
:105160005FC01124EECFCADFA0F3959FD1F3950F56
:1051700050E0551F629FF001729FBB27F00DB11DDB
:10518000639FAA27F00DB11DAA1F649F6627B00D6B
:10519000A11D661F829F2227B00DA11D621F739F54
:1051A000B00DA11D621F839FA00D611D221F749F62
:1051B0003327A00D611D231F849F600D211D822FA9
:1051C000762F6A2F11249F5750408AF0E1F08823F0
:1051D0004AF0EE0FFF1FBB1F661F771F881F9150FD
:1051E0005040A9F79E3F510570F014C0AACF5F3F11
:1051F000ECF3983EDCF3869577956795B795F79530
:10520000E7959F5FC1F7FE2B880F911D96958795B7
:1052100097F9089597F99F6780E870E060E0089536
:105220009FEF80EC089500240A94161617061806BE
:105230000906089500240A9412161306140605069A
:105240000895092E0394000C11F4882352F0BB0F2B
:1052500040F4BF2B11F460FF04C06F5F7F4F8F4F8E
:105260009F4F0895991B79E004C0991F961708F085
:10527000961B881F7A95C9F78095089597FB072E8E
:1052800016F4009407D077FD09D00E94582907FC36
:1052900005D03EF4909581959F4F08957095619546
:1052A0007F4F0895EE0FFF1F0590F491E02D0994B4
:1052B000AA1BBB1B51E107C0AA1FBB1FA617B7073C
:1052C00010F0A61BB70B881F991F5A95A9F7809558
:1052D0009095BC01CD010895F999FECF92BD81BD95
:1052E000F89A992780B50895A8E1B0E042E050E02F
:1052F0000C949429262FF999FECF92BD81BDF89A7E
:10530000019700B4021639F01FBA20BD0FB6F89409
:10531000FA9AF99A0FBE08950196272F0E947B29C9
:105320000C947A29DC01CB01FC01F999FECF06C06F
:10533000F2BDE1BDF89A319600B40D924150504053
:08534000B8F70895F894FFCFBF
:10534800FF790C6A0D470D130DDF0C0101CC012804
:1053580008140A321E796653436C49636F7F697378
:10536800091939293F4D362039FD04B0047A045A09
:105378000421049403AD03C603DF03FF0301020302
:085388000405060708090000F6
:00000001FF
